S026000062696E2F6F70656E626C745F6E75636C656F5F73746D33326631303372622E73726563D7
S3150800000000500020A5020008ED020008ED020008D5
S31508000010ED020008ED020008ED02000800000000ED
S31508000020000000000000000000000000ED020008CB
S31508000030ED02000800000000ED020008BD120008ED
S31508000040ED020008ED020008ED020008ED020008C6
S31508000050ED020008ED020008ED020008ED020008B6
S31508000060ED020008ED020008ED020008ED020008A6
S31508000070ED020008ED020008ED020008ED02000896
S31508000080ED020008ED020008ED020008ED02000886
S31508000090ED020008ED020008ED020008ED02000876
S315080000A0ED020008ED020008ED020008ED02000866
S315080000B0ED020008ED020008ED020008ED02000856
S315080000C0ED020008ED020008ED020008ED02000846
S315080000D0ED020008ED020008ED020008ED02000836
S315080000E0ED020008ED020008ED020008000000001D
S315080000F000000000000000000000000000000000F2
S3110800010000000000000000005FF808F195
S3150800010C10B5054C237833B9044B13B10448AFF337
S3150800011C00800123237010BD380400200000000065
S3150800012CF8170008084B10B51BB108490848AFF377
S3150800013C00800848036803B910BD074B002BFBD099
S3150800014CBDE81040184700BF000000003C04002022
S3150800015CF8170008380400200000000070B50F4E90
S3150800016C0F4D761BB61018BF002405D0013455F870
S3150800017C043B9847A642F9D10A4E0B4D01F036FBC3
S3150800018C761BB61018BF002406D0013455F8043B6C
S3150800019C9847A642F9D170BD70BD00BF6418000817
S315080001AC641800086C18000864180008024B13B190
S315080001BC024800F005B8704700000000D901000895
S315080001CC002301461A46184600F014B838B5074DF0
S315080001DC074C2C1BA41005D0013C55F8043D984738
S315080001EC002CF9D1BDE8384001F006BB70180008A0
S315080001FC6C1800082DE9F047254C064625688846F4
S3150800020CD5F8484192469946C4B360681F2817DC4E
S3150800021C411C76B104EB8003C3F888A0D4F8885146
S3150800022C012282401543022EC4F88851C3F808915E
S3150800023C1ED0831C6160002044F82380BDE8F0873B
S3150800024C144B03B34FF4C870AFF300800446D0B117
S3150800025CD5F84831002784E888003846C5F848415F
S3150800026C0121C4F88871C4F88C71002EE1D0D1E74D
S3150800027CD4F88C311A43C4F88C21DAE705F5A67440
S3150800028CC5F84841C1E74FF0FF30BDE8F08700BF1D
S3150800029C1018000800000000002103E00B4B5B5807
S315080002AC435004310A480B4B42189A42F6D30A4A71
S315080002BC02E0002342F8043B084B9A42F9D300F0BB
S315080002CCBDFBFFF74BFF00F087FC70477018000862
S315080002DC000000203804002038040020680900209B
S315080002ECFEE70000014B1860704700BF3004002081
S315080002FCC36813F4005F50D130B585B00D4604467B
S3150800030CC36823F4B05222F00C024968EB6819430F
S3150800031C2B690B431343C360AA68036923F4405340
S3150800032C134303616A69436923F4407313434361B6
S3150800033C684600F035F91C4B9C4201D1039B0AE038
S3150800034C1A4B9C4201D1029B05E0194B9C4201D1E8
S3150800035C029B00E0002313B3296811B303EB830354
S3150800036C03EB83038900B3FBF1F1124BA3FB0120CA
S3150800037C4009642202FB101212013232A3FB02233B
S3150800038CC3F34F1303F0F00202EB001003F00F0354
S3150800039C03449BB2A360012004E0002070470020B0
S315080003AC00E0002005B030BD003801400044004094
S315080003BC004800401F85EB51074AD36823F4E063D5
S315080003CC1B041B0C000200F4E060184340F0BF60ED
S315080003DC40F40030D060704700ED00E030B4164BA6
S315080003ECDB68C3F30223C3F10704042C28BF0424D7
S315080003FC1D1D062D01D9DD1E00E00025012303FA7B
S3150800040C04F4013C2140A940AB40013B1A400A4385
S3150800041C002806DA00F00F001201D2B2074B1A5464
S3150800042C07E01201D2B200F1604000F5614080F895
S3150800043C002330BC704700BF00ED00E014ED00E06F
S3150800044C0138B0F1807F0AD2064B5860F021064A73
S3150800045C82F823100020986007221A607047012042
S3150800046C704700BF10E000E000ED00E010B5064B49
S3150800047C4FF0FF32DA6000241C61DA60DC6000F0B1
S3150800048C17FC204610BD00BF0010024010B50446EC
S3150800049C0E4B18784FF47A73B3FBF0F30C4A1068CA
S315080004ACB0FBF3F0FFF7CCFF58B90F2C0BD8002292
S315080004BC21464FF0FF30FFF791FF064B1C600020DA
S315080004CC10BD012010BD012010BD00BF2C0400205A
S315080004DC300400202804002008B5074A136843F0A6
S315080004EC100313600320FFF767FF0020FFF7CEFF0A
S315080004FC00F07AFB002008BD00200240034B5B6825
S3150800050CC3F30313024AD35CD84070470010024069
S3150800051C14180008034B5B68C3F30223024AD35C26
S3150800052CD84070470010024024180008034B5B683B
S3150800053CC3F3C223024AD35CD8407047001002406A
S3150800054C241800080B4B5B6803F4803343B1094B42
S3150800055C5B6803F4003301330748B0FBF3F000E0A3
S3150800056C0648044B5B68C3F38343023303FB00F072
S3150800057C704700BF0010024000127A0000093D00C7
S3150800058C08B5054B5B6803F00C03082B02D1FFF783
S3150800059CD9FF08BD014808BD0010024000127A00B8
S315080005AC10B50446FFF7ECFF2060FFF7A7FF606065
S315080005BCFFF7B0FFA0606068FFF7B8FFE06010BDFA
S315080005CC264B98420BD103F58433DA6842F00402C1
S315080005DCDA60DA6822F00402DA6001207047204BF0
S315080005EC98420BD103F58233DA6842F00802DA60D6
S315080005FCDA6822F00802DA6001207047194B984233
S3150800060C0BD103F58033DA6842F01002DA60DA6847
S3150800061C22F01002DA6001207047134B98420BD176
S3150800062C03F57C43DA6842F02002DA60DA6822F0D5
S3150800063C2002DA60012070470C4B98420BD103F567
S3150800064C7843DA6842F04002DA60DA6822F040024F
S3150800065CDA60012070470020704700BF000801408F
S3150800066C000C014000100140001401400018014024
S3150800067CF0B583B00E68C6F30F2696FAA6F2B2FA50
S3150800068C82F26AE0012393401E4265D0072A03D8FA
S3150800069C40F20113934006E0A2F108044FF001134F
S315080006ACA34043F080634C681F0EC55993FAA3FE0A
S315080006BCBEFA8EFE4FEA8E0E4FF00F0C0CFA0EFE9B
S315080006CC25EA0E0E93FAA3F5B5FA85F5AD00AC40FE
S315080006DC4EEA0404C451C5681C0A25EA040E94FAA9
S315080006ECA4F4B4FA84F40D6905FA04F44EEA040485
S315080006FCC4604C68012C01D0092C2DD18C6801944E
S3150800070C93FAA3F5B5FA85F5AD004FF0030E0EFA7C
S3150800071C05F5C45924EA050E93FAA3F5B5FA85F539
S3150800072CAD00019CAC404EEA0405C551CC6893FA61
S3150800073CA3FEBEFA8EFE4FEA8E0E4FF0040C0CFA90
S3150800074C0EFE25EA0E0593FAA3F3B3FA83F39B0080
S3150800075C04FA03F31D43C551013236FA02F391D15B
S3150800076C012003B0F0BD00BF0022044BDA61044A35
S3150800077C136943F00103136101807047480900208F
S3150800078C002002401A4BDB6813F0100F06D0194AEA
S3150800079CD36943F00203D361102300E00023144A03
S315080007ACD26812F0040F06D01249CA6942F0010247
S315080007BCCA6143F004030E4AD26912F0010F09D03C
S315080007CC0C49CA6942F00402CA610949CA6922F08D
S315080007DC0102CA6140F20112934205D1044AD36957
S315080007EC23F00103D3617047014AD360704700BFF9
S315080007FC00200240480900200A4B1B6913F0800FA1
S3150800080C0BD0084B084A5A6002F188325A601B69A9
S3150800081C13F0800F03D10020704700207047012089
S3150800082C704700BF0020024023016745034A13693D
S3150800083C43F0800313610020704700BF002002407C
S3150800084C38B5044600F030FD054608E0B4F1FF3F24
S3150800085C05D024B300F028FD401B844221D3134B4A
S3150800086CDB6813F0010FF1D1104BDB6813F0200F86
S3150800087C02D020220D4BDA600C4BDB6813F0100FFC
S3150800088C09D10A4BDB6913F0010F04D1074BDB685E
S3150800089C13F0040F07D0FFF775FF012038BD0320AE
S315080008AC38BD032038BD002038BD00BF00200240EB
S315080008BC2DE9F843244C247E012C41D01E46904643
S315080008CC0F4604460122204B1A764CF25030FFF79D
S315080008DCB7FF034670BB012C04D0022C05D14FF090
S315080008EC020904E04FF0010901E04FF00409002465
S315080008FC1EE02101C1F12002A1F1200328FA01F121
S3150800090C06FA02F2114326FA03F3194389B207EBE6
S3150800091C4400FFF729FF4CF25030FFF791FF0B4BC1
S3150800092C1D6925F001051D61034618B90134E4B2A9
S3150800093C4C45DED30021044A11761846BDE8F883E7
S3150800094C0220BDE8F88300BF4809002000200240B9
S3150800095C0022064BDA61064B1A6942F004021A6148
S3150800096C1A6942F040021A61704700BF4809002014
S3150800097C002002400022064BDA61064B1A6942F047
S3150800098C02021A6158611A6942F040021A617047EC
S3150800099C4809002000200240264B1B7E012B47D01D
S315080009AC70B50E4605460122224B1A760368022BB1
S315080009BC12D14CF25030FFF743FF88BB0120FFF7EA
S315080009CCC7FF4CF25030FFF73BFF02461A490B693A
S315080009DC23F004030B6126E04CF25030FFF730FF8E
S315080009EC00BB4FF0FF333360AC68012211E02046A0
S315080009FCFFF7C0FF4CF25030FFF722FF0E4A13697F
S31508000A0C23F002031361024608B134600BE004F5C7
S31508000A1C8064E968AB6803EB81239C42E7D302E068
S31508000A2C012200E001220021024B1976104670BD06
S31508000A3C0220704748090020002002400F4B1A6814
S31508000A4C42F001021A6059680D4A0A405A601A683F
S31508000A5C22F0847222F480321A601A6822F48022F8
S31508000A6C1A605A6822F4FE025A604FF41F029A6002
S31508000A7C4FF00062034B9A60704700BF00100240AB
S31508000A8C0000FFF800ED00E0014B1880704700BF2E
S31508000A9C5804002008B500F0FFFB0E4B1B68984263
S31508000AAC16D30D4B1B7833B901220B4B1A70202227
S31508000ABC0A4B1A6105E00022074B1A702022074BD5
S31508000ACC5A6100F0E9FB064B1B881844014B186069
S31508000ADC08BD00BF540400205A0400200008014039
S31508000AEC580400202022014B5A6170470008014027
S31508000AFC08B5054B9B6813F4005F03D0FFF7F2FFAC
S31508000B0C012008BD002008BD0010014008B564206E
S31508000B1CFFF7BAFF08BD00BF08B5FFF7BBFF08BD56
S31508000B2C08B5264A136823F0070343F0020313603B
S31508000B3C136803F00703022B03D06821204800F042
S31508000B4CDBF8204B1A6842F480221A601A6842F4C1
S31508000B5C80321A601B4B1B6813F4003FFAD0194AF3
S31508000B6C536823F47C1343F4E8135360136843F077
S31508000B7C80731360134B1B6813F0007FFAD0114B6C
S31508000B8C5A6822F0F0025A605A6822F4E06242F47B
S31508000B9C80625A605A6822F460525A605A6822F087
S31508000BAC030242F002025A60064B5B6803F00C0320
S31508000BBC082BF9D10448FFF795FB08BD0020024025
S31508000BCC2C1800080010024000A24A0408B5FFF7CA
S31508000BDC83FCFFF7A5FF08BD08B5FFF7F7FF00F084
S31508000BEC97F800F0A3F8FCE7F0B58BB02D4B9A6993
S31508000BFC42F001029A619A6902F001020492049A7F
S31508000C0CDA6942F08052DA61DA6902F080520392AC
S31508000C1C039A9A6942F004029A619A6902F00402EC
S31508000C2C0292029A9A6942F010029A619A6902F043
S31508000C3C10020192019ADA6942F40032DA61DB6930
S31508000C4C03F400330093009B42F22003059301231F
S31508000C5C06930227079700260896134C05A92046E3
S31508000C6CFFF706FD2023636103F1846305930423D0
S31508000C7C069305A90D48FFF7FBFC40F204430593C0
S31508000C8C092506950797089605A92046FFF7F0FC4F
S31508000C9C40F608030593069505A92046FFF7E8FCD8
S31508000CAC0BB0F0BD001002400008014000100140D6
S31508000CBC08B50E48FFF784FC0D48FFF781FC0D4B71
S31508000CCCDA6922F40032DA619A6922F010029A6122
S31508000CDC9A6922F004029A61DA6922F08052DA6182
S31508000CEC9A6922F001029A6108BD00BF0010014002
S31508000CFC000801400010024008B500F005F8FCE7B2
S31508000D0C08B5FFF703FF08BD08B5FFF705FF08BDD3
S31508000D1C08B500F061FCFFF7F3FF00F09BFA00F052
S31508000D2C8DFC00F047F800F039F808BD08B5FFF758
S31508000D3CEBFF00F0A3FA00F049F800F001F808BD43
S31508000D4C08B500F081F8012813D00A4B1B78012B43
S31508000D5C0FD100F0A1FA084B1A68084B1B6813440C
S31508000D6C03F5FA73984204D30022024B1A7000F06A
S31508000D7C37FC08BD600400205C04002064040020D5
S31508000D8C08B5044B1B78012B03D100F085FA024BEE
S31508000D9C186008BD600400206404002008B5012210
S31508000DAC034B1A70FFF7ECFFFFF7CAFF08BD00BF2D
S31508000DBC6004002008B500F0B9F900F081FC0022A7
S31508000DCC014B1A7008BD00BF3404002000B583B06F
S31508000DDC0DF10701074800F0B1FC012807D10022E4
S31508000DEC054B1A709DF80710024800F0BDF903B0C0
S31508000DFC5DF804FB6804002034040020704700BF2B
S31508000E0C08B5044B1B7813B9C9B200F07BFC00F08B
S31508000E1CA3F908BD34040020044B1B78013B022BB4
S31508000E2C01D9402070470020704700BF34040020C9
S31508000E3C044B1B78013B022B01D94020704700203C
S31508000E4C704700BF3404002008B500F07DF900B1E6
S31508000E5C012008BD0022014B5A707047A8040020D7
S31508000E6C034BFE22DA7018710222A3F8442070474D
S31508000E7CA804002010B5054C00232370FFF7EAFFE1
S31508000E8CFF23E3700123A4F8443010BDA804002006
S31508000E9C064BFF22DA7000221A71597859719A7129
S31508000EACDA711A720622A3F844207047A8040020A7
S31508000EBC08B50020FFF7D4FF08BD00BF084BFF227A
S31508000ECCDA70084A9A6400221A715A719A710721C3
S31508000EDCD9711A725A729A720822A3F8442070476A
S31508000EECA804002034180008044BFF22DA70426864
S31508000EFC9A640122A3F84420704700BFA804002076
S31508000F0C08B53120FFF7ACFF08BD00BF38B5084C53
S31508000F1CFF23E370002525716571FFF77DFFA0712E
S31508000F2CE571257265720723A4F8443038BD00BFF5
S31508000F3CA804002038B5FFF78DFF0E4C0125257047
S31508000F4CFF23E3701023237100236371FFF764FFFB
S31508000F5CA071FFF76DFFE071FFF76AFFC0F307207A
S31508000F6C20726572A5720823A4F8443000F066FB5B
S31508000F7C38BD00BFA804002038B505464478FFF7ED
S31508000F8C4BFF0138844203DD2220FFF769FF38BD89
S31508000F9C084C6A78A16C201D00F040FBFF23E37017
S31508000FAC6B78A26C1344A3646B780133A4F84430B1
S31508000FBC38BD00BFA804002038B504464578FFF7AD
S31508000FCC2BFF0138854203DD2220FFF749FF38BD88
S31508000FDC6168084DA9646278281D00F01FFBFF2381
S31508000FECEB706378AA6C1344AB6463780133A5F889
S31508000FFC443038BDA8040020F8B505461746002429
S3150800100C06E015F8013B1C44E4B2FFF77DFE3146B9
S3150800101C4E1E0029F5D13C600120F8BD10B5084CD0
S3150800102CFF23E370E21D4168A06CFFF7E5FF207112
S3150800103C00236371A3710823A4F8443010BD00BFC4
S3150800104CA804002038B505460D4B9C6CFFF7E4FE4A
S3150800105C6A1C411E204600F0F5FA18B93120FFF734
S3150800106CFFFE38BD064CFF23E370FFF7D5FE0138AB
S3150800107CA36C1844A0640123A4F8443038BD00BFFF
S3150800108CA804002038B504464578FFF7C5FE023893
S3150800109C854203DD2220FFF7E3FE38BD0F4BFF2206
S315080010ACDA700122A3F84420617831B900F0DAFA33
S315080010BC90B93120FFF7D4FE38BDA21C074B986CAB
S315080010CC00F0C0FA18B93120FFF7CAFE38BD6378AC
S315080010DC024A916C0B44936438BD00BFA8040020E7
S315080010EC08B54168074B986C00F0B0FA18B931206E
S315080010FCFFF7B6FE08BD034BFF22DA700122A3F8F0
S3150800110C442008BDA804002008B500F069FA034B72
S3150800111CFF22DA700122A3F8442008BDA804002097
S3150800112C08B589B2FFF76CFE08BD00BF054B002257
S3150800113C1A709A6483F84320A3F844209A705A705C
S3150800114C704700BFA8040020024B187800B1012094
S3150800115C704700BFA80400200022024B83F84320E6
S3150800116C704700BFA804002008B50378FF2B02D1EE
S3150800117CFFF7E0FE50E0334A1278012A60D1C93BEA
S3150800118C352B46D8DFE803F03345454245453F360F
S3150800119C3C394545454545454545454545454545FA
S315080011AC45454545454545454545454545454545D5
S315080011BC4545241E1B2145454527452A2D30FFF755
S315080011CCDBFE29E0FFF7F8FE26E0FFF78DFE23E0AD
S315080011DCFFF724FF20E0FFF771FE1DE0FFF768FE1E
S315080011EC1AE0FFF755FE17E0FFF744FE14E0FFF789
S315080011FC29FF11E0FFF746FF0EE0FFF787FE0BE02D
S3150800120CFFF76EFF08E0FFF77FFF05E0FFF778FEB4
S3150800121C02E02020FFF724FE0A4B93F84330012BFB
S3150800122C02D11020FFF71CFE064BB3F94410002917
S3150800123C06DD1846012380F843300330FFF770FFAC
S3150800124C08BD00BFA80400200022014B1A60704795
S3150800125C10E000E008B5FFF7F7FF054B054A5A60A2
S3150800126C00229A6005211960034B1A6008BD00BF5D
S3150800127C10E000E03F190100F4040020044B1B6841
S3150800128C13F4803F03D0034A136801331360704785
S3150800129C10E000E0F404002008B5FFF7EFFF014B5F
S315080012AC186808BDF404002008B5FFF7F5FF08BD5B
S315080012BC704700BF08B5C1F3080353B903689942D0
S315080012CC09D040F8041B4FF4007200F0A7F901206E
S315080012DC08BD002008BD012008BD00BF2DE9F0415E
S315080012EC0746FFF789FA002413E03E68A30006EBCD
S315080012FC03083B445D68FFF707FD2A460023414671
S3150800130C0220FFF7D5FA40B956F824309D4206D18B
S3150800131C01347F2CE9D9012402E0002400E00024E2
S3150800132CFFF784FA2046BDE8F08100BF38B50D46B4
S3150800133C0B4B984207D004460A4B994205D0FFF747
S3150800134CCDFF18B908E0084C00E0054C29462046A4
S3150800135CFFF7B0FF10B938BD002038BD204638BDA0
S3150800136CF804002000200008FC0600202DE9F041B6
S3150800137C06460C4617461D4621F4FF7828F0010848
S3150800138C0368B3F1FF3F04D14146FFF793FF0346C9
S3150800139C30B33368984505D041463046FFF7C6FF4B
S315080013AC0646D0B13368E41A34440434FFF7ACFC6F
S315080013BC331DE31AB3F5007F07D308F500713046E1
S315080013CCFFF7B4FF064650B1041D17F8013B04F8A5
S315080013DC013B013DEAD1012302E0002300E0002392
S315080013EC1846BDE8F08100BF4FF0FF33024A136080
S315080013FC024A1360704700BFFC060020F804002060
S3150800140C10B54B1E114C241AA34218D8104B9842EF
S3150800141C17D90B18013B0D4CA34214D80B460146A1
S3150800142C20F4FF7020F001000A4CA04203D10A48B0
S3150800143CFFF79CFF10BD0948FFF798FF10BD002069
S3150800144C10BD002010BD002010BD00BFFFFF010815
S3150800145CFF1F000800200008F8040020FC060020E6
S3150800146C30B587B0002305934A1E1F4B1B1A9A42A8
S3150800147C32D820F47F7323F003031C4A93422DD9E8
S3150800148C0A18013A184CA2422AD8C01A0144C1F3C8
S3150800149C8F25C1F3090109B10135ADB200240194B8
S315080014AC039301230493FFF7A7F90CE0FFF72CFC31
S315080014BC05A901A8FFF770FA48B9039B03F58063E1
S315080014CC03930134A4B2A542F0D8012400E0002409
S315080014DCFFF7ACF9204604E0002002E0002000E00B
S315080014EC002007B030BD00BFFFFF0108FF1F000832
S315080014FC114B1B68B3F1FF3F18D000B583B00E4BE8
S3150800150C59689A681144DA6811441A6911445A6977
S3150800151C11449A691144DA698B185B4202AA42F89B
S3150800152C043D04210548FFF76BFF01E001207047D5
S3150800153C03B05DF804FB00BFF80400200C2100087A
S3150800154C0D4B1A6804331B6813440C4A126813446F
S3150800155C0B4A126813440B4A11680B44043212687E
S3150800156C1A44094B1B681344084A1268D34201D122
S3150800157C012070470020704700200008082000084A
S3150800158C0C20000810200008182000080C21000860
S3150800159C08B50D4B1B68B3F1FF3F04D00A48FFF79B
S315080015AC9DFE034668B1094B1B68B3F1FF3F05D096
S315080015BC0648FFF793FE034610B902E0012300E044
S315080015CC0123184608BD00BFF8040020FC060020BD
S315080015DC004870470020000808B500F003F908BD5C
S315080015EC10B500F037F8B0B1FFF782FA98B1FFF7EB
S315080015FC05FCFFF729FEFEF739FF00F02FF820F05F
S3150800160C604020F07F00044B986000F027F844688F
S3150800161C00F0EAF8A04710BD00ED00E070B508E050
S3150800162C461C4D1C0B780370FFF76EFB22463046A2
S3150800163C2946531E9CB2002AF2D170BD08B5FFF795
S3150800164CD3FE08BD08B5FFF7DBFE08BD08B5FFF7E6
S3150800165C07FF08BD08B5FFF773FF08BD08B5FFF708
S3150800166CB7FF08BD08B5FFF743FF034610B1FFF7F0
S3150800167C8FFF0346184608BD054B1B6813F0200F51
S3150800168C04D0034B5B680370012070470020704739
S3150800169C0044004010B5094B5860FFF7FDFD00F1FA
S315080016AC0A0405E0FFF730FBFFF7F6FD844204D386
S315080016BC024B1B6813F0800FF4D010BD0044004099
S315080016CC10B586B04FF4614300930023019302933F
S315080016DC03930C2204920593094C69462046FEF79F
S315080016EC07FE236923F490432361636923F02A03D5
S315080016FC6361E36843F40053E36006B010BD00BFB2
S3150800170C0044004070B506460D46402903D96F21A2
S3150800171C0948FFF7F1FA2846FFF7BCFF002406E054
S3150800172CFFF7F2FA305DFFF7B5FF0134A4B2ABB29E
S3150800173C9C42F5D370BD00BF3C18000870B5244B0D
S3150800174C1C78ACB92348FFF797FF01283ED1214BEB
S3150800175C1B78013BDBB23F2B38D8FFF79DFD1E4BA0
S3150800176C186000221D4B1A700122194B1A702DE0B5
S3150800177C06460D46194B1B78013316481844FFF7D5
S3150800178C7BFF0446012813D1144B1A780132D2B2C6
S3150800179C1A70104B1B789A4215D111493046FFF72F
S315080017AC3DFF00220A4B1A700C4B1B782B700DE070
S315080017BCFFF772FD084B1B686433984205D9002461
S315080017CC034B1C7002E0002400E00024204670BD88
S315080017DC4209002000090020440900204109002084
S315080017EC0109002072B6704762B67047F8B500BF9B
S315080017FCF8BC08BC9E467047F8B500BFF8BC08BCD8
S3090800180C9E4670472F
S315080018100000002000000000000000000102030490
S315080018200607080900000000010203046D61696EDD
S315080018302E6300004F70656E424C54002E2E2F2EDC
S315080018402E2F2E2E2F536F757263652F41524D43DF
S315080018504D335F53544D333246312F756172742EB2
S309080018606300000013
S30D08001864B90100083101000872
S3090800186C0D01000854
S3150800187000000000EC02002054030020BC030020F6
S31508001880000000000000000000000000000000004A
S31508001890000000000000000000000000000000003A
S315080018A0000000000000000000000000000000002A
S315080018B0000000000000000000000000000000001A
S315080018C0000000000000000000000000000000000A
S315080018D000000000000000000000000000000000FA
S315080018E000000000000000000000000000000000EA
S315080018F000000000000000000000000000000000DA
S3150800190000000000000000000000000000000000C9
S3150800191000000000000000000100000000000000B8
S315080019200E33CDAB34126DE6ECDE05000B0000007D
S315080019300000000000000000000000000000000099
S315080019400000000000000000000000000000000089
S315080019500000000000000000000000000000000079
S315080019600000000000000000000000000000000069
S31508001C900000000000000000100000000100000025
S30D08001CA000A24A04040000003A
S705080002A54B
